:10070B00416B6B756B6170617A69746165742020E4
:10071B0020002020202564206D416820202020000F
:10072B005369676E616C2062656920202020202050
:10073B0020202020200020202025642050726F7A5A
:10074B00656E7420200054454C4520456D666165EF
:10075B006E6765720056657273696F6E20312E304D
:10076B00002A004F4B2020202020200025322E3144
:10077B006641202020202020200025646D41682028
:10078B0020202020004665686C6572202000513DBA
:10079B0025332E316625252000FFFFFFFFFFFFFFCE
:1007AB0090FFFFFF91FF9293FFFFFFFF90FF909051
:1007BB0010FF91911192121393FFFFFF94FF9494EA
:1007CB0014FF95951596161797FFA8A828A9292AFF
:1007DB00AAAB2B2CAC2DADADFFFFFFFFAEFFAEAE2A
:1007EB002EFFAFAF2F98181999FF9A9A1A9BFF1BE0
:1007FB009B9C1C1D9D1E9E9EFFFF9F9F1FA020214B
:10080B00A1A22223A324A4A4FFA52526A627A7A73C
:10081B00FF30B0B0FFB0FFFFFFFFFFFFB1FFB1B183
:10082B0031FFB2B232B33334B4FFB5B535B6363768
:10083B00B7880809890A8A8AFFFF8B8B0B8C0C0DF2
:10084B008D8E0EFF8E0F8F8FFF80000181028282B3
:10085B00FF038383FF83FFFFFFFF8484048505066B
:10086B0086870738B839B9B9FFBA3A3BBB3CBCBC31
:10087B00FF3DBDBDFFBDFFFFFFBE3E3FBFFFBEBF88
:10088B00FFFFBEBFFFB9FFFFFFFFBEBFFFBCFFFFF8
:09089B00FFBDFFFFFFFFFFFFFF9F
:1008A400C103011200011600021A00000218000020
:1008B400011700C102010F00011400011300010817
:0108C40062D1
:10000E00E4FEFDEE25E0FEEF54014206EFC313FFC2
:07001E000DBD08EFAF062243
:10002500E4FDFCC3ED9FEC9E50070DBD00010C8067
:02003500F222B5
:10003700D2B712000E8F90D2B67F0A7E001200252B
:06004700C2B612002522E2
:10004D00C2B712000E8F90D2B67F0A7E0012002525
:06005D00C2B612002522CC
:0D0063007F0112004D7FE87E031200252270
:100070007FB87E0B120025C2B6C2B7E4F5907F3878
:1000800012004D7FE87E031200257F0C12004D7F89
:0A009000E87E03120025120063222F
:10009A008B308A318932AB30AA31A932120D89608C
:1000AA00127830E475F001120E54120D89FF120015
:0400BA003780E32286
:0F00BE00EF2480FFED75F040A42FFF12004D22BC
:1000CD0053073FD2A7D2A5D2A60DC2A6D2A5D2A6BE
:1000DD000DC2A6C2A5D2A60DC2A6E4FDEF30E50362
:1000ED00D38001C392A5D2A6EF25E0FFC2A60DBD18
:1000FD0006EAD2A5E4FDD2A6EB25E0FBEA33FAA28F
:10010D00A5E4334203E4C2A60DBD10EAC2A7AE02B8
:03011D00AF03220B
:1001200053073FD2A7D2A5D2A60BC2A6C2A5D2A67C
:100130000BC2A6D2A5D2A60BC2A6E4FBEF30E50304
:10014000D38001C392A5D2A6EF25E0FFC2A60BBBC8
:1001500006EAE4FBEC30E703D38001C392A5D2A604
:10016000ED25E0FDEC33FCC2A60BBB10E7D2A5C227
:10017000A6C2A7E4FB0BBB0AFCD2A7D2A6C2A6303C
:05018000A5FDC2A7224D
:10018500D2A5C2A6C2A7E4FFFE0FBF00010EEF6411
:100195000A4E70F5D2A7D2A5D2A6C2A6C2A5D2A6EE
:1001A500C2A6C2A5D2A6C2A6D2A5D2A6C2A6D2A5CD
:1001B500D2A6C2A6C2A7E4FEFF0FBF00010EEF64E0
:0501C5000A4E70F52256
:03000B000201CA25
:1001CA00C0E0C083C082C0D0C000C007A2B29204FF
:1001DA00D2B4E516C313F516300403431680200380
:1001EA001BE516B40F11D203AF140514744C2FF883
:1001FA0076FF53140F0513E4F51280370512E51242
:10020A00C39408402EE5169007A493B4FF13C203C3
:10021A00AF140514744C2FF8E4F653140F05138029
:10022A000FAF140514744C2FF8A61653140F0513A8
:10023A00E4F512E5176005D51702D283C2B4D007D8
:0B024A00D000D0D0D082D083D0E032B2
:03000300020255A1
:10025500C0E0C0D0858A15E515D394784005758C26
:1002650004800FE515C3946E5005758C08800375E1
:070275008C06D0D0D0E0326E
:10027C007F05AD1EAC1D1201207F06AD0EAC0D121C
:03028C000120222C
:10028F007F051200CD8E1D8F1E7F061200CD8E0DA5
:03029F008F0E229D
:1002A200E4F52FE52F14603C047070E4FFFD1200AA
:1002B200BE7BFF7A07790B12009AE4FF7D011200E0
:1002C200BE7533FF75340775351D851D36851E379E
:1002D2007B007A007968120FB47B007A0079681289
:1002E200009A8037E4FFFD1200BE7BFF7A07792B6C
:1002F20012009AE4FF7D011200BE7533FF753407C8
:10030200753541850D36850E377B007A0079681286
:100312000FB47B007A00796812009A20A2097F2C20
:100322007E0112002580F430A00F30A10C30A2090A
:100332007F2C7E0112002580EEE52F14601B0470D5
:100342002E20A008051EE51E7002051D20A120E535
:100352001E151E7002151D801620A008050EE50E42
:100362007002050D20A108E50E150E7002150D2074
:10037200A202052F7FE87E03120025E52FC3940217
:1003820050030202A512006312027C20A2097F2CF4
:080392007E0112002580F42217
:10039A00759852758922758869758DFD758C06D296
:1003AA008C75A883D28875B803120070120063E4B2
:1003BA00FFFD1200BE7BFF7A07795112009AE4FF13
:1003CA007D011200BE7BFF7A07796012009A120142
:1003DA008512028F20A2031202A230A00320A102DA
:1003EA00D202E51360EEAF0F050F744C2FF8E6F555
:1003FA002B530F0F1513B4FF16E4FFFD1200BE7B3B
:10040A00FF7A07796C12009AE4F508D20180C5E5F3
:10041A002B700E750863F50AF50CC2003001B58021
:10042A00B3E508146016146032240270A7E52B9015
:10043A0007A493543FF50B7508018098E52B9007A4
:10044A00A493543FF509C3940C400375090C75082D
:10045A0002E4F50AF50CC2000203DEE52B9007A4BC
:10046A0093543FFFAE0C050C74242EF8A607E50C36
:10047A00C3940450030203DEE5255403FFC4333357
:10048A0054C04524F528E526540FFFC454F0FFE56F
:10049A0025543CFE1313543F4FF529E5265430FFEB
:1004AA00C4540FFFE52725E025E04FF52AE4F52C93
:1004BA00E50A6509702BF52EF52DE52DC395095032
:1004CA000E745C252DF8E6252EF52E052D80EB748D
:1004DA0028252CF8E6652E60030206F6D2000206ED
:1004EA00F6E5092401FFE433FEE50A6F7001EE60C8
:1004FA00030206E8F52EF52DE52DC39509500C7477
:10050A005C252DF8E6622E052D80ED7428252CF841
:10051A00E6652E6003020667200003020667FF7D78
:10052A00011200BE7BFF7A07796E12009AC201059A
:10053A001BE51B7002051A785CE6F58008E6FE08E2
:10054A00E6FDEEF522EDF5237F01E4FD1200BE750E
:10055A0033FF753407753577AC22AD23EC120A6D7B
:10056A007B007A00792078411209CF8F398E388D35
:10057A00378C367B007A007968120FB4E4786FF60C
:10058A00FB7A00796812009A7F08E4FD1200BE78AF
:10059A005FE6FE08E6FDEEF522EDF5237533FF75FD
:0B05AA00340775358585223685233720
:1005B5007B007A007968120FB47B007A00796812A3
:1005C500009AC283751702AE0DAF0EEE3395E0FDAE
:1005D500FCF8F9AA06AB07AE1DAF1EEE3395E0FD9C
:1005E500FC120DE17B647A0079007800121446A8AC
:1005F50004A905AA06AB07AE22AF23EE3395E0FDAD
:10060500FCC3120E3E500A200270C2837517648027
:1006150069AE0DAF0EEE3395E0FDFCF8F9AA06AB19
:1006250007AE1DAF1EEE3395E0FDFC120DE17B64B8
:100635007A0079007800121446120E30A804A90534
:10064500AA06AB07AE22AF23EE3395E0FDFCD3122D
:100655000E3E400A200223C283751764801CC20225
:100665008018E4FF7D011200BE7BFF7A07799012A6
:10067500009A0519E519700205187F087D01120019
:10068500BE7533FF753407753599C3E51B9519FD9F
:10069500E51A9518FCE4120A6DC004C005C006C031
:1006A50007AC1AAD1BE4120A6DA804A905AA06AB8E
:1006B50007D007D006D005D0041209CF7B007A00F9
:1006C50079C878421208C68F398E388D378C367BBB
:1006D500007A007968120FB47B007A0079681200FD
:1006E5009A800E7428252CF8E6FF745C250AF8A676
:1006F50007050A052CE52CC3940350030204BAE44C
:06070500F50C0203DE22E8
:1008C600EC4D6011E8497017ED33EC3304600DE42C
:1008D600FCFFFEFD22E933E8330470F8020ADB125E
:1008E6000AA658046009E4CC24815006285009025F
:1008F6000AE5284003020AE2C0E0EB4A7044B980E8
:1009060006D0E0FB020AD1EF4E701CBD8008EBFF5B
:10091600EAFEE9FD80EBE98DF0A4FEE5F00209AF01
:10092600E9CDF9EAFEEBFFEF89F0A4FCE5F0CE890C
:10093600F0A42EFFE435F0CD89F0A42DFEE435F0C9
:100946008067EF4E7005BD80D780C3EF8BF0A4ACF7
:10095600F0EE8BF0A42CFCE435F0F8EF8AF0A42C32
:10096600E5F038FCE433CB8DF0A42CFCE5F03BF845
:10097600EE8AF0A42CFCE5F038F8E433CF89F0A435
:100986002CFCE5F038CF3400CE89F0A42FFFE5F03B
:100996003EFEE433C98DF0A42EFEE5F039CD8AF093
:1009A600A42FFFE5F03EFEE43DFD33D0E0FB50070B
:1009B6000BBB000F020AE5EC2CFCEF33FFEE33FE17
:0609C600ED33FD020ABD45
:1009CC00020AE5EC5D046005E859047003020ADBD9
:1009DC00120AA6580460F6EC4860F2EC7004FDFEB6
:1009EC00FF22C82481C85007C3985006020AE29817
:1009FC0050CEF582E9294B4A7005AB82020AD175BB
:100A0C00F0007C1A7880C3EF9BEE9AED99400DC3F1
:100A1C00EF9BFFEE9AFEED99FDE842F0DC23ACF083
:100A2C00D0E0FFD0E0FED0E0FDAB8220E7101BEB66
:100A3C0060BAEC2CFCEF33FFEE33FEED33FD020A13
:100A4C00BDE803F830E705C0F075F000EF2FFFEEBE
:0C0A5C0033FEED33FD40B830E7C280AA45
:100A680075F020800E75F010800575F0087D007E09
:100A7800007F003392D530D503120E30EC3340108E
:100A8800EF33FFEE33FEED33FDEC33FCD5F0ED2212
:0E0A9800E5F0247EA2D513CC92E7CDCEFF224E
:100F5800E5472433F8E60547227830300C02783329
:100F6800E475F001120E54020D892005EB7F2ED294
:100F7800058018EF540F2490D43440D4FF30090B67
:100F8800EF24BFB41A0050032461FFE5486002153E
:100F980048054BE54B7002054A300C0D7830E47576
:100FA800F001120E54EF020DCF02148A7403D20C12
:100FB8008003E4C20CF5478B308A318932E4F54866
:100FC800F54AF54BE54860077F20120F9380F5F549
:100FD80049C206C205C207C208C20AC20BC20D1224
:100FE8000F61FF700D300C057F00120FA4AF4BAEE0
:100FF8004A22B42563C2D5C209120F61FF24D0B4B6
:101008000A00501E75F00A20D50DC548A42548F5DC
:10101800487002D20880E0D205C549A42549F5499F
:1010280080D524CFB41A00EF5004C2E5D2090212C9
:1010380088D20680C2D20580BCD20780B8D2D580BB
:10104800B6D20A80B07F20120F932007077401B52B
:10105800480040F1120F58FF120F93020FCCD20D27
:10106800D20B8091120F58FB120F58FA120F58F931
:101078004A4B700679787A137BFF200733E548607E
:101088002FAF49BF00011F7E008E82758300120DAD
:10109800A260050EEE6F70F1C2D5EBC0E0EAC0E0C9
:1010A800E9C0E0EE1212E3D0E0F9D0E0FAD0E0FBBC
:1010B800120D89FF60A5EBC0E0EAC0E0E9C0E012CC
:1010C8000F93D0E02401F9D0E03400FAD0E0FBE53A
:1010D8004960DDD549DA8083D207809E1212C86044
:1010E800F7E549120AEFA949600BE54912136BEFBE
:1010F8007003D549F5EA30E702F404C3995077EA5A
:10110800F425490430E701E404F549800D1212C8BA
:1011180060C6EA05492549120AEFEA7846F630E73B
:1011280001E4254904D54904200A01141212E3E414
:10113800C0E012136B7846E6601320E70714F61236
:101148000F7B802204F6D0E014C0E07F00120F7BF2
:10115800E5496007120F721549800B300A03120F18
:1011680072D0E0020FCCD0E00480C51212C860A093
:10117800E54904120AEF7846EAF6E54904200A022E
:1011880060010424041212E374FF04C0E012136B1C
:10119800120F7BE549200A026003120F72D0E0B5F6
:1011A80049E87F45120F857846E67F2B30E7047FB4
:1011B8002DF404C0E0120F93D0E075F00A84C0F05B
:0311C800120F7C87
:1011CB00D0E0120F7C020FCC791080027908C20B91
:1011DB00C20D8008D2D5790A8004790AC2D5E4FA07
:1011EB00FDFEFF120F58FC7B08200613120F58FD53
:1011FB007B1030050A120F58FE120F58FF7B20ECA4
:10120B003382D592D55013C3E43005069FFFE49E7D
:10121B00FEE42006039DFDE49CFCE4CBF8C206EC47
:10122B00700CCFCECDCCE824F8F870F38017C3EF59
:10123B0033FFEE33FEED33FDEC33FCEB33FB994028
:10124B0002FB0FD8E9EB300605F8D0E0C448B20634
:10125B00C0E00AEC4D4E4F78207B0070C2EAC0E034
:10126B001212E5D0F0D0E0200604C4C0E0C4B206F0
:10127B00C0F0120F7CD0F0D5F0EB020FCC120E6445
:10128B00106C5311D358103D4C10394211D74F11DC
:10129B00DF4411DF4910524311E555111546117307
:1012AB004510E447139B5010412D10452E10682B11
:1012BB0010492310662013862A00001060100503C6
:1012CB00754906120F58FC120F58FD120F58FE12DB
:1012DB000F58FF783F020B1E790AA2D52008143055
:1012EB000A09B910020404B9080104A2D5200B02A3
:1012FB005001042007669207B548005032C0E07FCA
:10130B00203008177F30A207720B720A500D121390
:10131B003AC207C20BC20A7F30800F300A03E9C002
:10132B00E0120F93300A03D0E0F9D0E0B548CE308D
:10133B000A177F30B9100C120F937F583009077FB3
:10134B00788003B90803120F933007057F2D020F26
:10135B00937F20200DF87F2B200BF322920780CF59
:10136B007F00B407005005243FF8E6FF22286E7576
:10137B006C6C29002D50434958D206120F58300679
:10138B00F8C206784830D504D2057849F6020FFD2D
:10139B00120F582403B405004001E490137F9312FD
:0F13AB000F84743A120F84D2087548040211D3CC
:100AA600E9D2E7C933E833F892D5EDD2E7CD33EC96
:070AB60033FC5002B2D5220F
:100ABD00EC30E7100FBF000C0EBE00080DBD00049A
:100ACD000BEB6014A2D5EB13FCED92E7FD2274FF46
:100ADD00FCFDFEFF22E480F8A2D574FF13FC7D809F
:020AED0080F097
:100AEF00F920E72824F950037907E4F42402FB18CE
:100AFF00DBFDE624FB5014E9600DE4F618E604F67E
:0F0B0F00B40A08E4F6D9F57401F60A22C2D52219
:100B1E00ED33EC3392D5FA602AB4FF33EDC2E77BA6
:100B2E00FF60067A0B7943E4227A0B794C20D504C8
:100B3E007A0B7947224E614E002B494E46002D49C5
:100B4E004E4600E47A08F608DAFC7B00740722E8C9
:100B5E00C0E0ECC0E0EDC0E0EEC0E0EFC0E0EA7552
:100B6E00F010A4CAABF075F04DA42BFBE435F0FCED
:100B7E00EA2410FAEB34C5FBEC34D9FCEDC2E7FFE6
:100B8E0075F056A4F42411C5F0F434C58FF0A42AE0
:100B9E00E5F03BE43CF620E714120D49D0E0FFD01F
:100BAE00E0FED0E0FDD0E0FC1209CF8014F4041278
:100BBE000D49D0E0FFD0E0FED0E0FDD0E0FC120801
:100BCE00C6D0E0F8E6FAEDD2E7CD33EC332482FB63
:100BDE00E4C3CF33CFCE33CECD33CD33DBF37B0770
:100BEE0075F00A846004F6081B0AE5F0F6088FF02B
:100BFE00740AA4FFACF08EF0740AA42CFEACF05074
:100C0E00010C8DF0740AA42CFDE435F0F608DBDE41
:030C1E0074072236
:100C2100020ADBE86480F8E933E83360110460F01C
:100C3100ED33EC337009E8FCE9FDEAFEEBFF220439
:100C410060DED3EB9FEA9EE99DE8C2E78CF0C2F734
:100C510095F0400CE8CCF8E9CDF9EACEFAEBCFFB00
:100C6100120AA685D0F05804700320D5B3E80470A9
:100C7100075002B2D5020AE592D5EC0460F7E4CC44
:100C8100C0E0C398F8603B94186008400DD0E0FBC9
:100C9100020ABDE4FBFAC9FC8028E830E406E4C995
:100CA100FBE4CAFCE830E305E4C9CACBFCE854071D
:100CB1006010F8C3E913F9EA13FAEB13FBEC13FC28
:100CC100D8F130F52FC3E49CFCEF9BFFEE9AFEEDCB
:100CD10099FDD0E0FBEF4E4D4C701222DB03020A6E
:100CE100E2EC2CFCEF33FFEE33FEED33FDED30E7AC
:100CF100EB020ABDEF2BFFEE3AFEED39FDD0E0FB32
:100D010050130BBB0003020AE5ED13FDEE13FEEFDA
:080D110013FFEC13FC020ABD04
:100D19003F8000004120000042C80000447A0000E2
:100D2900461C400047C35000497424004B18968064
:100D39004CBEBC205A0E1BCA6753C21C749DC5AE5B
:100D4900FB60065407601C2323120D77EB543860AF
:100D590009120D63120D721208C6ECF8EDF9EEFADC
:100D6900EFCB22EB120D7280F1543803241C900D45
:100D790019FE93FC0EEE93FD0EEE930ECE93FF2219
:030000000213BA2E
:0C13BA00787FE4F6D8FD75817B021401F9
:100D8900BB010689828A83E0225002E722BBFE0268
:090D9900E32289828A83E493229B
:100DA200BB010CE58229F582E5833AF583E0225006
:100DB20006E92582F8E622BBFE06E92582F8E22250
:0D0DC200E58229F582E5833AF583E493226A
:100DCF00BB010689828A83F0225002F722BBFE0103
:020DDF00F322FD
:100DE100E88FF0A4CC8BF0A42CFCE98EF0A42CFCB1
:100DF1008AF0EDA42CFCEA8EF0A4CDA8F08BF0A42F
:100E01002DCC3825F0FDE98FF0A42CCD35F0FCEB8D
:100E11008EF0A4FEA9F0EB8FF0A4CFC5F02ECD3952
:0F0E2100FEE43CFCEAA42DCE35F0FDE43CFC22BF
:10144600C2D5E830E70FB2D5E4C39BFBE49AFAE4D1
:1014560099F9E498F8EC30E717B2D512147C120E1D
:10146600C6E4C39BFBE49AFAE499F9E498F880038E
:10147600120EC630D50DE4C39FFFE49EFEE49DFD2B
:04148600E49CFC22C4
:0E0E3000C3E49FFFE49EFEE49DFDE49CFC22D3
:100E3E00EB9FF5F0EA9E42F0E99D42F0EC6480C82B
:060E4E0064809845F022CB
:100E5400FAE6FB0808E6F925F0F618E6CA3AF6229F
:100E6400D083D082F8E4937012740193700DA3A31D
:100E740093F8740193F5828883E473740293686031
:060E8400EFA3A3A380DF31
:10148A00EFB40A07740D121495740A309811A899CA
:10149A00B8130CC2983098FDA899C298B811F630C2
:0714AA0099FDC299F599229A
:1013C60002039AE493A3F8E493A34003F68001F2A0
:1013D60008DFF48029E493A3F85407240CC8C33328
:1013E600C4540F4420C8834004F456800146F6DFF7
:1013F600E4800B01020408102040809008A4E47EDB
:10140600019360BCA3FF543F30E509541FFEE493EB
:10141600A360010ECF54C025E060A840B8E493A3B2
:10142600FAE493A3F8E493A3C8C582C8CAC583CADD
:10143600F0A3C8C582C8CAC583CADFE9DEE780BE95
:0108C5000032
:100E8A0075F008758200EF2FFFEE33FECD33CDCC1F
:100E9A0033CCC58233C5829BED9AEC99E5829840A2
:100EAA000CF582EE9BFEED9AFDEC99FC0FD5F0D67F
:100EBA00E4CEFBE4CDFAE4CCF9A88222B800C1B9A9
:100ECA000059BA002DEC8BF084CFCECDFCE5F0CBE7
:100EDA00F97818EF2FFFEE33FEED33FDEC33FCEB20
:100EEA0033FB10D703994004EB99FB0FD8E5E4F9DB
:100EFA00FA227818EF2FFFEE33FEED33FDEC33FCC8
:100F0A00C933C910D7059BE99A4007EC9BFCE99ABB
:100F1A00F90FD8E0E4C9FAE4CCFB2275F010EF2F00
:100F2A00FFEE33FEED33FDCC33CCC833C810D70700
:100F3A009BEC9AE899400AED9BFDEC9AFCE899F83B
:0E0F4A000FD5F0DAE4CDFBE4CCFAE4C8F922CE
:00000001FF
